:030000000219FDE5
:03000B000200AA46
:03002B0002015679
:03005B000202E9B5
:030073000202CFB7
:1000800002030406080C10182030406080040608A3
:100090000C10182030406080A0C000070F1F3F0DDB
:1000A0000D04050D050305030302C2AFC0D0C0E077
:1000B000206217E5256002E473E525F4F58A758B67
:1000C00000D262D0E0D0D0D2AF3285268AC262E5BB
:1000D00026F46035306803207210758B00D0E0D0B4
:1000E000D0D295D293D297D2AF32D295D293D29723
:1000F000206E0C206609740CD5E0FDE57E429075FB
:100100008B00D0E0D0D0D2AF32758A00C28DD262DF
:1001100001FF01B9306805206602C29501B9306857
:1001200005206602C29701B9306805206602C293B5
:1001300001B9C294306805206602C29501B9C29621
:10014000306805206602C29701B9C2923068052066
:100150006602C29301B9C2AFC2AD53E6EFC0D0C0D0
:10016000E0D2D3D2AFC2CEE52A6007207449152A67
:1001700021B77800790020742EE580307E01F430BC
:10018000E50278FF53DACF207E0343DA20307E0386
:1001900043DA10C2D8C271E580307E01F430E50246
:1001A00079FFC3E89970CB306103752A1820740376
:1001B000752A18885FD27020740DE52B6004152B0A
:1001C00021C743DA01C2D82070024125A85F20610F
:1001D00002C2702074367982B70431C3E894F040CB
:1001E0000374F0F8E8C4540F28F87984B703024187
:1001F0000CC313C3138721200802C313200A06C3AC
:10020000C898F8410C28F8500374FFF88822E52DAF
:1002100054066011E533C313C31324062522F522C7
:1002200050037522FF7882B60459852224A824C37E
:10023000E52495644002A864C3E895664002A86678
:100240008825E56970024176C3E8AA699A5003E8F7
:10025000FAE4F9EAC333FBE56BF45B29400D256A48
:10026000F8E56A6002156A400B41760AC3E56A9AAE
:100270005002056A78FF8826C26EC3E52694F840CE
:1002800002D26EC3E52594404002D26420CF0AD04A
:10029000E0D0D043E610D2AD32C2CF053A7801E5C6
:1002A0002A6005307402152AC3E55F940140057584
:1002B000620041C5756300756C00E5622401F5625A
:1002C00050037562FFD0E0D0D043E610D2AD32C209
:1002D000AFC0D053E67FC2607591008556948557B4
:1002E00095759104D0D0D2AF32C2AF53E6EFC2AD14
:1002F000C0D0C0E0C0F0D2D3D2AFA8FBA9FCC2D816
:10030000307102615053DACF207E0343DA10307E21
:100310000343DA20D271E580307E01F420E50261EA
:100320002788278928A17753DACF207E0343DA2054
:10033000307E0343DA10C2D8C271307402A16378F0
:1003400000E580307E01F430E502A163885FA14BB7
:1003500053DACF207E0343DA20307E0343DA10C223
:1003600071206102812953DACF207E0343DA1030F5
:100370007E0343DA20C2D8D271885A895BC3E895DC
:1003800058F8E99559F97B007E087A00C3E8948C07
:10039000E994005005755E00811B882178A2E6A8CB
:1003A000216055C3E894C8E994005008E4D2E4FB06
:1003B0007A0A61F6C3E89468E994015008E4D2E34C
:1003C000FB7A0F61F6C3E894D0E994025008E4D2B6
:1003D000E2FB7A1E61F6C3E894A0E994055008E4B4
:1003E000D2E1FB7A3C61F6C3E89498E9940850089E
:1003F000E4D2E0FB7A787E00C3E8955CFCE9955D89
:10040000FD30E70AECF42401FCEDF43400FD755EE8
:1004100000C3EC9AED9E5003755E01885C895D8592
:100420005A58855B597802A14BC3E89527F8E9959E
:1004300028F9307C02A12F307B02A12F307A02A153
:1004400028207502814CE9FDE8FC816BE9C313F9B2
:10045000E813F8307902A128E9C313F9E813F8305A
:100460007802A128E9C313FDE813FC206126C3EC40
:0E047000941CED940240028182ED7018C3ECE2
:10047E0094C850120529C3E529940A5002A1637548
:10048E005F00D270A163E529600215297888E6F92C
:10049E007400207F087896B90302789EE624FAFE4F
:1004AE00E43400FFC3EC9EFCED9FFD9208B90310EF
:1004BE00A2085007207609D27681CE307602C27617
:1004CE00A2085016B9030DECF42401FCEDF434002F
:1004DE00FD0204E878007900A12FB90315EC33FC76
:1004EE00ED33FDC3EC940AFCED9400FD50047C004A
:1004FE007D00C3EC94FFED9400400678FF7900A1D7
:10050E002FEC8575F0A4C5F0A2F733F879004003FF
:10051E0002054B78FF790002054BE9C313F9E81386
:10052E00F8307C0EE9600278FFC3E81338F8E43443
:10053E0000F9C3E894FFE99400400278FF885FD287
:10054E0070206102A163741FF4552F4BF52FC274F6
:10055E00EB7002D274752A18307403752A0A306152
:10056E0002A17720740353DAFE207403752B06D094
:10057E00F0D0E0D0D0D2AD43E6103279010205A71B
:10058E0079030205A7790A0205A7791E0205A77944
:10059E00640205A779C80205A77817E4D5E0FDD84F
:1005AE00FAD9F6227A147B780205CE7A107B8C0269
:1005BE0005CE7A0D7BB40205CE7A0B7BC80205CE32
:1005CE007902B27DE4C296D5E0FDC297D5E0FDD2A8
:1005DE0097D5E0FDD296D5E0FDC295E576D5E0FD46
:1005EE00D2957496D5E0FDD9D9EAF8D5E0FDD8FBC1
:1005FE00DBCEC29622C37C007D0075F00005F0EACA
:10060E0033FAEB33FB50F6EB13FBEA13FAC3E9FFB5
:10061E00E8FEE89AF8E99BF95004EFF9EEF8B3EC2E
:10062E0033FCED33FDD5F0DFEDF9ECF822E889F07F
:10063E008A20D2D4F8A9F07B0030F70B7BFFF4248C
:10064E0001F8E9F43400F9E88520F0A4ADF0F8E9FA
:10065E008520F0A4AFF0FEED2EF974003FFA7C0475
:10066E00C3EA13FAE913F9E813F8DCF48BF030F768
:10067E000AE8F42401F8E9F43400F9E889F0C2D468
:10068E00F8A9F0227882B604030206EDC3E55F9462
:10069E000140030206B7852224E4F545F546F547E9
:1006AE00F548F549C26D0206ED7882E6FCD26DE59D
:1006BE0022F523783879C7AA40AB41C3EB13FBEA86
:1006CE0013FAEC146013C3EB13FBEA13FAEC1414D5
:1006DE006007C3EB13FBEA13FAD103884589462260
:1006EE00C3E5459523F8E5469400F9500CC3E8940C
:1006FE0080E994FF401602071EC3E8947FE9940038
:10070E00500302071E787F790002071E788079FF5A
:10071E00884A894B22E54A2547F8E54B3548F98545
:10072E004B20E4300701F43549FA30E709C3EA9467
:10073E00F0401502075CC3EA940F500302075C7881
:10074E00FF79FF7A0F02075C780079007AF0C3E533
:10075E00249564500AC374019524500B02077AE560
:10076E004B20E70E02077AE54B30E70688478948AB
:10077E008A492278A4E6FAC3E54A33F8E54B33F901
:10078E00D13BE930E70BC3E89480E994FF4013E1D5
:10079E00B4C3E8947FE994005002E1B4787F790005
:1007AE00E1B4788079FFE820E715C3E52398F84097
:1007BE0009C3E8940140030207DB78010207DBE876
:1007CE00F424012523F840030207DB78FF884C222E
:1007DE0078A5E6FAA848A949D13BE930E70CC3E869
:1007EE009401E994FF401602080FC3E894FFE994C0
:1007FE0000500302080F78FF790002080F78017984
:10080E00FFE920E715C3E54C98F84009C3E89401C9
:10081E0040030208367801020836E8F42401254C1C
:10082E00F8400302083678FF88242278FFC264203D
:10083E00693D206A12D264C3E541940A4009C3E5BA
:10084E002594405002C26479A1E76023E541601F00
:10085E0074FF8541F0848539F0306A0375F005A484
:0F086E00F8C5F0600278FFC3E895675002A867ED
:10087D00886622C3E5409440E5419401E566500346
:10088D00140191046002F566220208992275E89020
:10089D00227883E6FFE5E820ECF7A8BDA9BE057335
:1008AD00C3E57394084052757300E9FA79A0E760C7
:1008BD0044EA7007E574601B0208D4C3E8957460C0
:1008CD0010E5745006600C140208E00460F902088B
:1008DD00E0E574F574C3946D401B7564C0C3940456
:1008ED004013756480C39404400B756440C3940435
:1008FD00400375640075BB0822E564241050027432
:10090D00FFF5647982B70402212DC3A864E524980C
:10091D005002A824C3E895664002A866882588265B
:10092D00E573B4070375BB1022743279A687F0A462
:10093D00C5F0A2F733F8C3E895644002A864882295
:10094D008824882588268867227540007541F02205
:10095D00C2AF75C820A8CCA9CDAA3A30CF010A756F
:10096D00C824D2AFAB3BAC3C883B893CC3E89BF879
:10097D00E99C206908F9306702417221CFAD3D8AAB
:10098D003DF9EA9DFA600478FF79FFAE3EAF3F8BEB
:10099D003E8C3FC3EC9FFCC3E99CF542A83BA93CB0
:1009AD00C3E89EF8E99FF9C3E54113FBE54013FA4F
:1009BD00E82AF540E93BF54150067540FF7541FFCA
:1009CD004119AA40AB41AC40AD417E047F02C3EB5F
:1009DD00940440021E1FC3EB940840021E1FC3ED7A
:1009ED0013FDEC13FCDEF7C3EA9CFAEB9DFBEF6005
:1009FD0009C3E913F9E813F8DFF7EA28FAEB39FB35
:100A0D008A408B4150067BFF8B408B41C3EB940298
:100A1D005002D2673069047F0341447892E6FFC3E8
:100A2D00E537948240110FC3E53794A040010FC301
:100A3D00EF940640027F057E05E541C4540FF9E5AC
:100A4D0041C454F0F8E540C4540F28F8C3E89EFAA9
:100A5D00E99400FB4009C3EA9402EB940050047A38
:100A6D0002E4FB41BEAA40AB41EBC4FEEAC4540F05
:100A7D004EFCC3EA9CFAEB9400FBC3E813C313F8D6
:100A8D00EA28FAEB3400FB8A408B41C3EB94024019
:100A9D0002C2677805EBC4FE7B00EAC4540F4EFA20
:100AAD00C3EA98FA4005C3940250027A027892E69E
:100ABD00FF30600241BE855256855357D26043E6E2
:100ACD0080C3E49AF8E49BF93067026158E8FAE9CB
:100ADD00FBD3E913FDE813FC88528953C3EF94034C
:100AED006038EF20E00DE82CF8E93DF9ECFAEDFB6C
:100AFD00020B13E828F8E939F9C3E82402F8E934C0
:100B0D0000F97AFE7BFFC3EF9403400E8A548B5598
:100B1D00884E894F8C508D51618C885489558A4EE1
:100B2D008B4F8C508D51306920C3E53394034019A0
:100B3D00E542A2E713F8E555F4240138400B20E710
:100B4D00087554FFF42401F555618CE8FAD3E813C8
:100B5D00FC8852C3EF94036020EF20E007E82CF8E7
:100B6D00ECFA6178E8282402F87AFEC3EF9403408A
:100B7D00088A54884E8C50618C88548A4E8C50E56E
:100B8D006BC3335002646BF56B3060026196753444
:100B9D0002D26043E680E52D54066026A840A941A7
:100BAD00C3E913F9E813F8C2AF53E67F759100C39B
:100BBD00E498F594E499F595759104D26043E68037
:100BCD00D2AF22D265754400752000306B037520BD
:100BDD0040020BEFD265754400752040306B0375F4
:100BED002000D2AF7801206722E52D54066002C2A5
:100BFD0065C3E541940540137802940540087803D8
:100C0D00940540027806306902780A206019E5449F
:100C1D00601530690AC3E53394034003D53406D219
:100C2D00AFD26C81C0719ED2AF0000C2AF206726DB
:100C3D00E541C3FB940F40027B0FEB24053073019C
:100C4D0023306A02742820620123F9306902798207
:100C5D00E58BC39940B50544E59B5440B520028111
:0E0C6D00AA30690A08C3E8940A4001088118F9
:100C7B0020650261EFC26553E67F75910030671006
:100C8B007594007595FE759104D26043E68061EF13
:100C9B00AE40AF41C3E49EF594E49FF5958191C3BB
:100CAB00E5339402500261EF30650261EFD80281A7
:100CBB00BE8118C26C53E67F75910085549485559F
:100CCB0095759104854E56854F57D26043E680D279
:100CDB00AFE52D54066008206A020533020CFA308A
:100CEB006C0D206B0A206507158115810215652295
:100CFB0078003064053065027801E53775F007A49C
:100D0B00F9E5F028F5F0E9A2F013A2F113A2F21322
:100D1B00F537C394785003753778C3E5379538406A
:100D2B0008D266D295D293D297306002A134855007
:100D3B0056855157D26043E68022207D11C2AF7594
:100D4B004302C296D294D2AF759F11020F14C2AF59
:100D5B00754302C296D292D2AF759F11020F143017
:100D6B007243207D20C2AF75430390013E757E40D8
:100D7B00D293C292306204C297A188D296D2AF7539
:100D8B009F13020F14C2AF75430390013E757E4053
:100D9B00D295C294306204C297A1A8D296D2AF75F5
:100DAB009F10020F14207D17C2AF75430390011ED5
:100DBB00D293306202C297D2AF759F13020F14C247
:100DCB00AF75430390011ED295306202C297D2AF2A
:100DDB00759F10020F14207D11C2AF754304C2948E
:100DEB00D292D2AF759F10020F14C2AF754304C2DB
:100DFB0092D294D2AF759F13020F14307243207DA1
:100E0B0020C2AF754305900132757E10D297C29602
:100E1B00306204C295C124D294D2AF759F11020FD8
:100E2B0014C2AF75430590014A757E04D297C296E2
:100E3B00306204C293C144D292D2AF759F11020F9C
:100E4B0014207D17C2AF754305900114D297306201
:100E5B0002C295D2AF759F11020F14C2AF75430535
:100E6B00900128D2973062EBC293D2AF759F1102DB
:100E7B000F14207D11C2AF754306C292D296D2AF2A
:100E8B00759F13020F14C2AF754306C294D296D24C
:100E9B00AF759F10020F14307242207D20C2AF75C8
:100EAB00430190014A757E04D295C294306204C20C
:100EBB0093C1C0D292D2AF759F10020F14C2AF75FF
:100ECB004301900132757E10D293C292306204C2FC
:100EDB0095C1E0D294D2AF759F13E114207D16C259
:100EEB00AF754301900128D295306202C293D2AF05
:100EFB00759F10E114C2AF754301900114D293306A
:100F0B006202C295D2AF759F13C266229001127511
:100F1B007E00D295D293D297C294C292C296C262ED
:100F2B0022788076090876090876040876FF087619
:100F3B00030876FF08760A0876030876010876011F
:100F4B00788C76010876FF0876FF0876FF0876FF27
:100F5B000876FF0876030876FF0876FF0876FF0809
:100F6B0076250876D0087628087650087604087619
:100F7B00FF08760208760008767A0876FF08760175
:100F8B00087601087600087603227887E6FFC2729E
:100F9B00BF0302D2727888E6C394036008C27DE671
:100FAB0030E102D27DC27E7889E630E102D27EC387
:100FBB00EF94026008758E01D273020FCD758E000F
:100FCB00C273227880E6149000809378A4F678811F
:100FDB00E6149000809378A5F67886E61490008D41
:100FEB009378A6F6789CE67538FF75390CB4020633
:100FFB007538A075390AB4030675388275390578CA
:10100B00A3E61490009A93F569120F172222789693
:10101B00E6FA7897E6FB7888E6B40305C3EB940E03
:10102B00FB307F047A007BFFC3EB9AFCC3948250A6
:10103B00027C827575000575EC8575F0A4C3E5F02F
:10104B00947D40F222D27F11191205987A007B0011
:10105B007C1012058EE55F2AFA74003BFBDCF37CF7
:0F106B0004C3EB13FBEA13FADCF7FEC27F111983
:10107A0022E5EF20E6037520000520903FFFE520DA
:10108A00146006901DFF1460009304600375EF124C
:10109A0053D9BF7581C043FF8012058975EF02439A
:1010AA00B203E5B3240420E70DF521E5E320E006C9
:1010BA008521B343E301120F177580FF75A40075EC
:1010CA00F1B275D4DF7590A975A5FC75F2FE75D5D8
:1010DA000175A60175E241E4F8F6D8FD756B0112B7
:1010EA000F2C1215A778988676753001C2AF1205B3
:1010FA00A21205B21205981205B91205981205C076
:10110A00120598C2AF78FA79FA308507D9FBD8F771
:10111A00021C00120F95120FCE1118111978988619
:10112A0076120F1775885075891275C8247591043F
:10113A0075D84075A82275B80275E690759B8075BA
:10114A009D0075D10E75BC5875BB0875BA1175E846
:10115A0080120589D2AF12089653DACF207E034354
:10116A00DA20307E0343DA1043DA01C2D8C27112A0
:10117A0005A2D2617B037A0CE55E70077A0CDB0369
:10118A0002110D12059820700302110DC270E55F5D
:10119A00C3940240E1E52F541F856160F561B56093
:1011AA00D5DAD5C26153DACF207E0343DA20307E06
:1011BA000343DA10C2D8C27178A2E67008D274E585
:1011CA002F54E0F52FC27575290012059D30740958
:1011DA00C3E529940A4002D27512058E780230744A
:1011EA00027800C3E55F9840F0C2AF1205B212055B
:1011FA00B21205B2D2AF1205A2754D007888E6B4D4
:10120A00030241E412058E788CE6C394015003026E
:10121A0012E4E530C3940150030212E4207435C38A
:10122A00E55F94FF50030212E4C2AF1205C7D2AFC2
:10123A0012059DC3E55F940150EFC2AF1205B212C9
:10124A0005931205B2D2AF12059DC3E55F94FF4024
:10125A00E902174F7F02D27F111912059DC2AFC250
:10126A007F1119AE5FC3E55F947FD2AF4076120556
:10127A0089C2AF1205C7D2AFDFDC1150C3EE9405A5
:10128A007897F61205A21215E91216D27F0AD27FB2
:10129A00111912059DC2AFC27F1119AE5FC3E55F76
:1012AA00947FD2AF50E6120589C2AF1205B2120579
:1012BA00931205B2D2AFDFD61150EE24057896F616
:1012CA001205A21215E912170112059D1119C3E59B
:1012DA005F94FF5002412602174FC3E55F954D40C8
:1012EA0003855F4D12059D78017988E7B40302787A
:1012FA0005C3E55F9840024106C2AF1205C7120551
:10130A00C71205C7D2AF1205A2753000E4F531F550
:10131A00320531E531F470390532789AE6781914D4
:10132A006012783214600D787D14600878FA1460BF
:10133A0003753200C3E53298401715327531B47817
:10134A00998676C2AF1205C7D2AF7898867612050B
:10135A009D120593E52A7005307402210D7801204B
:10136A0074027806C3E55F9840A77888E6C39403B9
:10137A00600312059DE52A700302110DC2AF120F18
:10138A0017E4F522F523F524F525F526F56AD2AFFB
:10139A007885E6C333F568E4F545F546F547F5483B
:1013AA00F549F573F52CF52DF53775730875BB10EE
:1013BA0012058912089AE5E820ECFBA8BDA9BEE946
:1013CA007001F8887412089E75730875BB107887C7
:1013DA00E6FE7602120F957887EEF6C2AF7564FFC5
:1013EA00120936852264852265852266D2AF752266
:1013FA000175240175250175260185636C756D01DA
:10140A007888E6B40307C27D307602D27DD268D2EC
:10141A0069753300120E7D120EA212095612095D69
:10142A0012095612095D120956021443C2AF120F6D
:10143A0095D2AF75730075BB08120BE112069212B2
:10144A000CFB120D4512095D120BD0306D0312060A
:10145A00EE206703120839306703120880120CFB6A
:0F146A00120D6A12095D120BE1306D0312072398
:10147900120CFB120DE112095D120BD0306D031233
:101489000781120CFB120E0612095D120BE1306D79
:10149900031207DE120CFB120E7D12095D12089A67
:1014A900120BD0120CFB120EA212089E12095D300B
:1014B9006935206B3285676485676585636C756DF1
:1014C9000179187A0CC3E53399400FC269D26A8A47
:1014D900358567648567660214F0C3E55F9401404A
:1014E9000302144302156D306A1B206B18E535148D
:1014F9007004C26A8136F535C3E55F940140030281
:10150900144302156D753600C3E56278FA98505494
:10151900307404E52A604D7888E6B40317207D0508
:10152900207607A13D307602A13D206B07D26B855D
:101539006764818278F0306B058567647820C3E53C
:10154900419850028143306B1BC26BC27D307602D9
:10155900D27DD26A75351285676481430536E55FA8
:101569006002A170753600C2AF120F177887E6FEC8
:101579007602120F957887EEF6E4F522F523F52425
:10158900F525F526F568C268D2AF120589120F173D
:10159900307409C3E53694054002210D6116901A8D
:1015A9000D782012162BE520B4550CA312162BE545
:1015B90020B4AA030215C9120F2C1215E90215E865
:1015C900901A0378807B0A12162BA308DBF9901A6C
:1015D9000F788C7B1812162BA308DBF9901A272297
:1015E900C2AF12166A121644901A00740E121630FF
:1015F900A37404121630A37414121630901A0378C7
:10160900807B0A12162FA308DBF9901A0F788C7BBE
:101619001812162FA308DBF912167D12165B901A01
:101629002722E493F622E6438F01538FFD75EF02DB
:1016390075B7A575B7F1F0538FFE22438F02438F1B
:101649000175EF0275B7A575B7F1901A0DF0538FB3
:10165900FC22901A0D7455D130901A0E74AAD1300B
:10166900227A3079D07820901A40D12BE520F709D9
:10167900A3DAF7227A3079D0901A40E7D13009A35A
:10168900DAF922AB77A878BB01027980BB0202792B
:1016990081BB03027982BB04027984BB0502798686
:1016A900BB06027992BB07027987BB080279A3BB03
:1016B9000902799CBB0A027988BB0B027989E8F790
:1016C900227C051205A2DCFB22C2AF1205B212056B
:1016D900B91205C01205C71205931205B21205B950
:1016E9001205C01205C71205931205B21205B912E7
:1016F90005C01205C7D2AF22C2AF1205C71205C075
:101709001205B91205B21205931205C71205C012C6
:1017190005B91205B21205931205C71205C01205C3
:10172900B91205B2D2AF22AE77AF78C2AF1205B205
:101739001205B21205B2120593DEF21205C712059F
:1017490093DFF8D2AF22D1D2D1CAD1CA7577017548
:101759007801757900F1307C05AD5F1205A2C3ED02
:10176900955F70F5C3E55F9401400AC3E55F94FF97
:10177900403202178BD18CB1E9D1D2C2AF75EF12C9
:10178900D1CADCD50579C3E5799403500280C6D165
:10179900CA0578E5771490009F93F808C3E578980F
:1017A900500280AED1CAD1CA0577C3E577940C50EF
:0F17B90002809C120F2CB1E9C2AF75EF12D1CA9A
:0319FD0002107B5A
:101A00000E0414090904FF03FF0A03010155AA018A
:101A1000FFFFFFFFFF03FFFFFF25D0285004FF0259
:081A2000007AFF01010003FF41
:101A400023526F746F724765656B73323041232088
:101A500023424C48454C4923463333302320202031
:101A60002020202020202020202020202020202076
:101C0000C2AFC2D353D9BF7581C043B20343FF8073
:101C1000752438752503B1C975EF0275E24043F1AB
:101C20002053A4DF75D400D2857DFA780379E67C51
:101C300010752200752300901DD67B0675249875BB
:101C400025013085028142208508D8FBD9F9DCF7CF
:101C500081B4308508D8FBD9F9DCF781B4B189E4C7
:101C600093A3C39A6004DDC381B4DBDBB17B600264
:101C7000812B7B08E493FAA3B15CDBF87A30B15C8A
:101C8000752200752300B17BEAFCEBFDC3ED94FEE9
:101C9000400EB17B8A278B28ED30E0048A828B834B
:101CA000B17B7AC270D8C3ED94FE601350CEBD00F4
:101CB00025EC60097520007521FF0200008100A855
:101CC00027A9280809D804D90281D3B17FEA89AAB3
:101CD000F281C50D81A0C3ED94035049EDA2E092BD
:101CE000007AC5C3E5829400E583941C50902000DF
:101CF00010438F02438F0175B7A575B7F1F030001F
:101D00001FA827A9280809438F01538FFDD804D99C
:101D100002A12089AAE275B7A575B7F1F0A3A10DBC
:101D2000538FFC817C7AC1BD030CE493A3FAB140CC
:101D3000DCF8B138817C817EAA22AB23B15CEBFA5E
:101D4000EA6222752608C3E52313F523E52213F57D
:101D50002250066323A0632201D526EAB1C9B1C986
:101D600075260AEAF4200102D285300102C285B14B
:101D7000C9C3134002C201D526EB22B17FEAFB2082
:101D80008502A17F308502A184752608AE24AF2587
:101D9000C3EF13FFEE13FEB1CDB1C9C3EA13308513
:101DA000024480FA30E703632201C3E52313F523DD
:101DB000E52213F52250066323A0632201D526D91C
:101DC000E52265236523F52222AE24AF250E0FDE22
:101DD000FEDFFCD20122424C48656C693437316326
:041DE000F3300601D5
:00000001FF
